:1003BC005452414E5A005354414E44414C4F4E45B9
:1003CC00000000112332465765748C9DAFBECADB0A
:1003DC00E9F810013322564775649C8DBFAEDACB19
:1003EC00F9E82130021367764455ADBC8E9FEBFAC9
:1003FC00C8D93120120377665445BDAC9E8FFBEAF9
:10040C00D8C94253617004152736CEDFEDFC8899AC
:10041C00ABBA5243716014053726DECFFDEC9889D8
:10042C00BBAA6372405125340617EFFECCDDA9B888
:10043C008A9B7362504135241607FFEEDCCDB9A8B8
:10044C009A8B8495A7B6C2D3E1F008192B3A4E5F6C
:10045C006D7C9485B7A6D2C3F1E018093B2A5E4F98
:10046C007D6CA5B48697E3F2C0D129380A1B6F7E48
:10047C004C5DB5A49687F3E2D0C139281A0B7F6E78
:10048C005C4DC6D7E5F48091A3B24A5B69780C1D2C
:10049C002F3ED6C7F5E49081B3A25A4B79681C0D58
:1004AC003F2EE7F6C4D5A1B082936B7A48592D3C08
:1004BC000E1FF7E6D4C5B1A092837B6A58493D2C38
:1004CC001E0F0089129B24AD36BF48C15AD36CE570
:1004DC007EF78108931AA52CB73EC940DB52ED6418
:1004EC00FF76028B109926AF34BD4AC358D16EE704
:1004FC007CF5830A9118A72EB53CCB42D950EF66F8
:10050C00FD74048D169F20A932BB4CC55ED768E1E3
:10051C007AF3850C971EA128B33ACD44DF56E960D7
:10052C00FB72068F149D22AB30B94EC75CD56AE3C3
:10053C0078F1870E951CA32AB138CF46DD54EB62B7
:10054C00F97008811A932CA53EB740C952DB64EDB3
:10055C0076FF89009B12AD24BF36C148D35AE56C97
:10056C00F77E0A8318912EA73CB542CB50D966EF83
:10057C0074FD8B029910AF26BD34C34AD158E76E77
:10058C00F57C0C851E9728A13AB344CD56DF60E963
:10059C0072FB8D049F16A920BB32C54CD75EE16857
:1005AC00F37A0E871C952AA338B146CF54DD62EB43
:1005BC0070F98F069D14AB22B930C74ED55CE36A37
:0B05CC00F178FF03BCFF03C2FF03CD6A
:0319DF000176008E
:101924009001F2E06FFC9004CE93FE9001F0E0FD94
:10193400EE6D9001F2F0AF04EF9003CE939001F0BE
:01194400F0B2
:01194500227F
:10000300C2AFC28E758900438910758BE0758DC1AF
:07001300D2ABD28ED2AF2266
:03001B0002177554
:10177500C0E0C0D0C28E758BE0758DC1201B06758B
:10178500A61E75A6E10576D218E57C6002057C05E6
:101795007FE57F540F7020D223E57F543F7002D23E
:1017A50014E57BD394014002157BE57ED394644018
:0E17B50004D21B8002057ED28ED0D0D0E0324E
:030023000212A81E
:0B12A800C0E0C083C082C0D075D01829
:1012B300309850757C01AF99201709EF6402704193
:1012C300D217803D301F04C21F8024BF0904D21FE0
:1012D300802FBF02055378808027BF03129000221E
:1012E300E578F0637840537840C217D21A801274BD
:1012F3006F2578F582E43401F583EFF005785378B0
:101303007FC298309964C29930165F9000A6E0FFBF
:101313009000EDE0D39F400DC216D220201D02D2D3
:1013230021C21D80459000EDE0FF04F074EE2FF51F
:1013330082E43400F583E0F57D301C16537D7F3065
:10134300152520D00520191F800330191A637D80CD
:101353008015301512E57D527D301906A2D0929B7F
:0C1363008005A2D0B3929B857D99D2AF8B
:09136F00D0D0D082D083D0E0324E
:10187500C216C221C21AC217C21FE49000EDF09031
:1018850000A6F0F578F57CC21CD220E579F5CBE50C
:0E1895007AF5CA85CBCD85CACCD29CD2AC22C6
:0610F1007E007F007D027D
:0210F700A90549
:1010F900E49001F0F09001F2F08E4E8F4F9000EEE7
:101109007402F0E4FB7A01EBC3995051854F828553
:101119004E83E0FF121924854F82854E83E024FD1A
:10112900600824FA600424077010AF020A74EE2FD5
:10113900F582E43400F5837409F0054FE54FAE4EAE
:101149007002054E14F5828E83E0FFAE020A74EE3A
:101159002EF582E43400F583EFF00B80AA9001F2BA
:10116900E0FF24FD600824FA600424077010AE0231
:101179000A74EE2EF582E43400F5837409F0AE02A8
:101189000A74EE2EF582E43400F583EFF09001F055
:10119900E0FF24FD600824FA600424077010AE0201
:1011A9000A74EE2EF582E43400F5837409F0AE0278
:1011B9000A74EE2EF582E43400F583EFF074EE2A1A
:0C11C900F582E43400F5837403F0AF02FB
:0111D50022F7
:10180A00E49001F0F09001F2F0900022E05440FBE5
:10181A00900022E0FFEBC39F5012746F2BF582E415
:10182A003401F583E0FF1219240B80E49001F0E003
:0B183A00FF9001F2E04F7002C322D3C8
:011845002280
:10003600C2AF1217C3D2AFC2221211D6121875C29E
:100046001B120003C2AFE49001F1F0757B01D2AF41
:1000560075A70775A61E75A6E1020352302323C2B3
:10006600239001EFE0600B14F0E07006E577600284
:1000760015779001F3E0600214F09001F1E0600260
:1000860014F0E4F57E201E030202321207CF900020
:10009600A7E024FE700302019214700302021814F2
:1000A60070030201C91470030201F0240470AD123A
:1000B60018469000A8EFF06003020189900022E044
:1000C600700302016212180A50030202B090002265
:1000D600E0FF5440FEF54DFD054D746F2DF582E4AD
:1000E6003401F583E09000A5F0E0B4FE04C2AF80D1
:1000F600FEAD4D054D746F2DF582E43401F583E0B8
:1001060090016EF0EF543FFFD394044044746F2E79
:10011600F582E43401F58363A20190002463A20111
:10012600EF14FF12103D900022E0543F24FCFF9094
:1001360000A4F01219679000A7500B7404F0900108
:10014600F37414F080137405F09001F3740FF080CB
:1001560008E49001EFF075770A0202B09001F1E031
:1001660060030200627425F0121378302203020045
:10017600629000A5E090020CF0A374FDF09000A838
:100186007414F09000A77402F002006230160302A5
:100196000062E49001F0F09001F2F07E027F0C9094
:1001A60000A8E0FD1210F79000A6EFF0E49000ED35
:1001B600F0D216D2999000A704F09001EF7406F0E1
:1001C6000200629000A4E0FF121967400F9000A79A
:1001D6007405F09001F3740FF00200629001F3E0F1
:1001E6006003020062C2AF020062120026EF6016D0
:1001F6009000A5E0900000F090016EE0900001F004
:100206009000A77403F09001F3E06003020062021D
:10021600037E3016030200621210F19000A6EFF082
:10022600E49000EDF0D216D29902037E900023E00E
:1002360024FE606814700302038614700302035AD6
:100246002403600302006230220E121946D21E9069
:1002560000A77401F00200623016030200629000EB
:100266000074FEF0A374A0F0A37431F0A3742EF012
:10027600A37430F0A3F07E007F007D061210F79085
:1002860000A6EFF0E49000EDF0D216D2999000238C
:100296007402F09001EF740AF0020062900022E00E
:1002A600700302034912180A5008E4900022F00273
:1002B6000062900022E0FF5440F54DFE054D746F3C
:1002C6002EF582E43401F583E09000A5F0746F25E5
:1002D6004DF582E43401F583E090016EF0EF543F72
:1002E600D3940A403DE064907038F54D7424254D52
:1002F600F582E43400F5837420F0054DE54DB480B5
:10030600EB900022E0FF54402471F582E43401F5BD
:100316008363A20190002463A201EF543F14FF12ED
:10032600103DE4900022F090016EE0B4900C12199A
:10033600469000237404F00200629000237403F0D8
:100346000200629001EFE060030200629000230465
:10035600F0020062301603020062121A0B8F4D7E05
:10036600027F0CAD4D1210F79000A6EFF0E490005E
:10037600EDF0D216D299D21E9000A704F0020062C8
:100386003016030200629000A5E0900000F0900194
:100396006EE0900001F01210F19000A6EFF0E490EC
:1003A60000EDF0D216D2999000237402F09001EF7E
:0603B600740AF00200626F
:1011D600E4F54EE54E75F003A424CEF582E434051D
:1011E600F583E493FB740193FA740293F91205D71D
:1011F60070030212A7E4F550F551F54F7424254FFC
:10120600F582E43400F583E0FF70030212A2E54E96
:1012160075F003A424CEF582E43405F583E493FB4C
:10122600740193FA740293F985508275830012054E
:10123600F0FEEFB506077551010550805AE551607D
:1012460056EE704EE54E1460450470507424254FDA
:10125600F9E43400FA7B01C0031B8B59755A0075FB
:101266005B00E4F55CD00312097F8F558E548D53D5
:101276008C52AB55AA54A953A8527FB07E717D0BF0
:101286007C001206591206EB8E798F7A800ED222D6
:10129600800AE4F551F550054F021202054E02117F
:0112A600D96E
:0112A7002224
:1014D20042415544004E4F5F4D45414E44520057E4
:1014E2005F4D4F44454D00534C415645004C4541DC
:1014F20044455200494E565F52454300494E565F9D
:101502005452414E5300494E565F414C4C0000C864
:10151200CCDF73696E7573625F6772616E69742E78
:1015220062696E00312E3000C4C0D2C030382F3014
:10153200332F30390031323A35353A313300FF1426
:10154200D2FF14D7FF14E1FF14E9FF14EFFF14F6E2
:10155200FF14FEFF1508FF15100008040C020A060E
:091562000E0109050D030B070F32
:1019E2005201F800000000000000000000000000AA
:0519F2000000000000F0
:061A0B00900310E0FF2231
:100CC100E4900310F0E0FF04F0740C2FF582E4349B
:100CD10002F58374FEF0900310E0FF04F0740C2F12
:100CE100F582E43402F5837491F0900310E0FF047F
:100CF100F0740C2FF582E43402F5837430F0900324
:100D010010E0FF04F0740C2FF582E43402F58374D3
:100D11000DF0900310E0FF04F0740C2FF582E43421
:100D210002F583740AF0E4FFEFC39404501EEF90C0
:100D3100152693FE900310E0240CF582E43402F5AD
:100D410083EEF00F900310E004F080DCE4FFEFC3CA
:100D51009415501EEF90151493FE900310E0240C8F
:100D6100F582E43402F583EEF00F900310E004F015
:100D710080DCE4FFEFC3940D501EEF90152E93FE1F
:100D8100900310E0240CF582E43402F583EEF00FB9
:100D9100900310E004F080DC900310E0FF04F07495
:100DA1000C2FF582E43402F5837420F0E4FFEFC3E5
:100DB1009409501EEF90153793FE900310E0240C18
:100DC100F582E43402F583EEF00F900310E004F0B5
:100DD10080DC900310E0FF04F0740C2FF582E43402
:100DE10002F583740AF0900310E0FF04F0740C2FF5
:090DF100F582E43402F583E4F01C
:010DFA0022D6
:1019880090030EE06FFC9004CE93FE90030FE06E80
:0F19980090030EF0AF04EF9003CE9390030FF087
:0119A700221D
:02166C008F5697
:10166E00900310E0240CF582E43402F5837420F02C
:10167E00900310E004F0E4FFEFC39D503BE5567578
:10168E00F003A42440F582E43415F583E493FB744F
:10169E000193FA740293F98F827583001205F0FE9E
:1016AE00900310E0240CF582E43402F583EEF00F83
:0816BE00900310E004F080C06D
:0116C6002201
:1018FB0074242FF582E43400F583E0FE6420601835
:10190B00900310E0240CF582E43402F583EEF00F23
:08191B00900310E004F080D8F5
:0119230022A1
:100B2300E4F54EE54E75F003A42440F582E4341554
:100B3300F583E493FB740193FA740293F91205D7D6
:100B43007003020CC0E4F550F551F54F7424254FA2
:100B5300F582E43400F583E0FF7003020CBBE54E3D
:100B630075F003A42440F582E43415F583E493FB84
:100B7300740193FA740293F9855082758300120508
:100B8300F0FEEFB506087551010550020CB6E551AC
:100B93007003020CB6EE6003020CB1AD50AF4E12FF
:100BA300166CE54EB408004003020CBB900BB6F87C
:100BB300282873020BCE020C62020C66020C9B0205
:100BC3000C9F020CA3020CA7020CABAF4F1218FB35
:100BD3007424254FF9E43400FA7B01C0031B8B59BD
:100BE300755A00755B00E4F55CD00312097F8F55DD
:100BF3008E548D538C52E4FFFEFDFCAB55AA54A9D1
:100C030053A852C31206F9601FAB55AA54A953A89F
:100C130052E47F847E1EFDFC1206591206EB9003FC
:100C230014EFF0E4900313F0E47F587E02FDFCAB75
:100C330055AA54A953A852D31206F9407B90031323
:100C43007401F0AB55AA54A953A8527F487EE8FD1E
:100C53007C001206591206EB900314EFF08059D270
:100C6300038055AF4F1218FBD2107424254FF9E4BB
:100C73003400FA7B01C0031B8B59755A00755B0066
:100C8300E4F55CD00312097F8F558E548D538C523B
:100C930090020AE555F08020D213801CD20E8018F2
:100CA300D20B8014D2088010D20BD208800AE4F54C
:0D0CB30051F550054F020B4F054E020B2668
:010CC0002211
:1019F800EF540F90155B93C454F0FEEFC4540F934B
:031A08002EFF228C
:101846003012299000A5E090020CF090016EE09015
:10185600020DF090028E63A20190020E63A201E5D2
:0F1866007324FEFF12103DC212AF73227F0022C7
:10171F008F75C225E4FFE56D64056030E575B47E15
:10172F0002802EE57530E707436801056D8006538B
:10173F0068FEE4F56D056FE56FB40808856870D233
:10174F0025E4F56FE56825E0F568800DE57530E770
:10175F0005D204A22522E4F56DE57525E0F5750F98
:05176F00BF08B3A22534
:011774002252
:0715F700E0FF1219F8C22504
:1015FE00E4FEE56E25E0F56EEF30E736436E012032
:10160E002533056DE56DB4052CE4F56D0572E572B7
:10161E00B40817056CE56CAC6B7002056B14F582A3
:10162E008C83E56EF00574E4F572E56E25E0F56EDB
:10163E008003E4F56D0572E572B40817056CE56C70
:10164E00AC6B7002056B14F5828C83E56EF005743D
:0D165E00E4F572EF25E0FF0EEE64087095D4
:01166B00225C
:1018D100754B7E7544A0C206D20DC212D224C2112C
:1018E100C201C221D200C20FC296C297E49000A5E4
:0A18F100F090016E7408F00218A3D5
:1019460090031474B8F0E4900313F090031204F0BB
:10195600120CC1120B231216C71218D1C297C296C7
:01196600225E
:10142F00E4F574900317F0A3F0A3F0AB07AA0675C9
:10143F006B02756CCE856C82856B83747EF0056C48
:10144F00E56C7002056B0574E4F572900315F0906E
:10145F000315E0C39D50498B828A83E0FF1219F870
:10146F00900316EFF0900319E06F900316F0E0FF72
:10147F009004CE93FE900318E06EA3F0EF9003CE8E
:10148F0093900318F00BEBAE0270010A14F5828EE5
:10149F0083E0FFC2251215FE900315E004F080AF24
:1014AF009003191215F79003181215F7D2257F7EA6
:1014BF001215FED225E4FF1215FED201756B0275CF
:0214CF006CCEE1
:0114D10022F8
:10196700AD0720011A900025E0FF64026004EFB480
:1019770008097E007F2612142F8002D221C322D3AA
:01198700223D
:101378007F020F740C2402F582E43402F5837408AA
:10138800F00F740C2403F582E43402F583E4F07C56
:10139800017DFDFEED1DAA0470011CF5828A83E023
:1013A800FBAA070F740C2AF582E43402F583EBF0EC
:1013B8000EBE04E07C027D01E4FEED1DAA0470016E
:1013C8001CF5828A83E0FBAA070F740C2AF582E4D5
:1013D8003402F583EBF00EBE04E07C027D05E4FEEA
:1013E800ED1DAA0470011CF5828A83E0FBAA070F91
:1013F800740C2AF582E43402F583EBF00EBE04E0A7
:101408007C027D09E4FEED1DAA0470011CF5828AA8
:1014180083E0FBAA070F740C2AF582E43402F583F3
:06142800EBF00EBE04E033
:01142E00229B
:100DFB00200603020EBFE542543865397003020F1B
:100E0B0002E53924085438F539131313541F2429D8
:100E1B00F8E6F570200429FF12171F50D9AF701296
:100E2B0019F8121988056AE56AAE6970020569142A
:100E3B00F5828E83E570F00573E573D3948040B62D
:100E4B00C206D212C204D224C29690030EE0FFA3B4
:100E5B00E04F603EC212900202E0FCA3E0FDA3E073
:100E6B00FEA3E02401FFE43EFEE43DFDE43CFC90E8
:100E7B00020212070A90028EE07002D20290031156
:100E8B00E004F0D394055003020E01D202E4F00209
:100E9B000E019001FAE0FCA3E0FDA3E0FEA3E02429
:100EAB0001FFE43EFEE43DFDE43CFC9001FA120739
:100EBB000A020E01202440E529647E7022300205CF
:100ECB00D224C20222D200D296D206E4F573F56D7B
:100EDB0090030EF0A3F0F56F756902756A8E22E52B
:100EEB0029B4A01120050ED20090028C7402F0A33D
:070EFB0074EEF0C207D224DF
:010F020022CC
:1007CF00201E05D296D2972230180AC21890020B1B
:1007DF00E0600214F0300D03120DFB20110302082C
:1007EF006DE543653A6048E54324085438FFE53A20
:1007FF0054386F60047E0180027E00E57460047DD2
:10080F000180027D00EE5D700302097E056CE56CD0
:10081F00AC6B7002056B14F5828C83E0FEE543131D
:10082F001313541F2431F8A6068F43157480B8C2D2
:10083F0097C211C2019001FEE0FCA3E0FDA3E0FE10
:10084F00A3E02401FFE43EFEE43DFDE43CFC900107
:10085F00FE12070AD221D2B2E490020BF022300628
:10086F000302097E30014FE543653A600302097EBA
:10087F0030B208C2B290020AE0A3F030100C3090F0
:10088F000990020BE0600302097E056CE56CAE6B0C
:10089F007002056B14F5828E83E0FFE5431313138B
:1008AF00541F2431F8A607E54324085438F543159F
:1008BF0074D211D29722E543653A600302097E3064
:1008CF00030302097E30B208C2B290020AE0A3F01D
:1008DF0030100C30900990020BE0600302097E206B
:1008EF00001F900206E0FCA3E0FDA3E0FEA3E024BE
:1008FF0001FFE43EFEE43DFDE43CFC9002061207DE
:10090F000AC200E54324085438F543131313541F48
:10091F002431F876AAE54324085438F5431313130A
:10092F00541F2431F876A0E54324085438F54313B7
:10093F001313541F2431F8E4F6E54324085438F513
:10094F0043131313541F2431F8E4F6E543240854DA
:10095F0038F543131313541F2431F8E4F6E54324F9
:10096F00085438F543131313541F2431F8E4F622B7
:0B002600302105C2217F01227F002253
:1016C700C2A9438902900314E0FFF58C8F8A75D96C
:1016D7000475DC4975DD4975DA31E4F5E9F5F9F5A5
:1016E700EBF5FB900313E0601675EC1075ED10E455
:1016F700F5FCF5FD754108753B10754001801375C4
:10170700EC8075ED80E4F5FCF5FD754180F53B75E2
:081717004010E4F5EAF5FA22A6
:1018A300E4FE900314E0658C60041216C70EE5D9BC
:1018B30020E2057E021216C7E58920E1051216C74C
:0D18C3007E03D28C75D840D2AED2AFAF06F6
:0118D00022F5
:03003300020F03B6
:070F0300C0E0C0D075D0086A
:100F0A00C2AF30D82AC3E5EC95EAC39541500DE546
:100F1A004025ECF5EC30D71205FC8011C3E5EC95C1
:100F2A0040F5EC30D70415FC800385FCFCC2D830B0
:100F3A00D902C2D930DA67E53B700405FC8010E5B6
:100F4A003B25ECF5EC30D70405FC800385FCFCE579
:100F5A00275480F54CE52725E0F52730930205272D
:100F6A00200B03632701302419E527654B6006E54A
:100F7A002765447027753900754200852729C224E0
:100F8A00801A0542E5425407701253423FE5421364
:100F9A001313541F2429F8A627752700C2DA30DB59
:100FAA0049E53B700405FD8010E53B25EDF5ED3084
:100FBA00D70405FD800385FDFDE543653A6029E513
:100FCA003A54077013E53A131313541F2431F8E601
:100FDA00F5282008036328FFE528339292E528259F
:0C0FEA00E0F528053A533A3FC2DBD2AFD5
:050FF600D0D0D0E03274
:100FFB00740093F8ECC3984024701F740193F8EDC0
:10100B00C39840197014740293F8EEC398400E7095
:10101B0009740393F8EFC39840037F00227F0122EA
:10102B00EDF8E6F008A3DFFA22EDF8E0F608A3DF0F
:10103B00FA22E0A363A201F0A363A201DFF475A27D
:10104B000022E0A363A2016DFE936CFDEE0583937A
:10105B00FC158363A201DFEA75A200227F00E493F3
:10106B00A363A201F00F600CA3E583C2E3F58363D6
:10107B00A20180EA75A20022E0A363A201F0A3E51E
:10108B0083C2E3F58363A201DFEE75A20022E0A326
:10109B0063A201F0A3E583C2E4D2E3F58363A2016B
:1010AB00DFEC75A20022E583C2E3F583E0A363A224
:1010BB0001F0A363A201DFEE75A20022E583C2E477
:1010CB00D2E3F583E0A363A201F0A363A201DFECFB
:0F10DB0075A20022F922C002C004C00612FFF065
:0710EA00D006D004D0022261
:1019A800E5D220E0FBC2AF438E2075D2028F82754C
:0C19B8008300E0FFE4F5D2538EDFD2AFD5
:0119C4002200
:1019C500E5D220E0FBC2AF43D2028F82758300EDE2
:0A19D500F075D25063D250D2AF2259
:1017C300E4FEEE247FFF1219A874242EF582E4347C
:1017D30000F583EFF074242EF582E43400F583E002
:1017E300701B74242EF582E43400F5837420F074A6
:1017F300252EF582E43400F583E4F080040EBE80E8
:06180300C1E49000A3F017
:0118090022BC
:0300000002156B7B
:0C156B00787FE4F6D8FD75817F0215B290
:1005D700BB010689828A83E0225002E722BBFE0222
:0905E700E32289828A83E4932255
:1005F000BB010CE58229F582E5833AF583E02250C0
:1006000006E92582F8E622BBFE06E92582F8E22209
:0D061000E58229F582E5833AF583E4932223
:10061D0075F008758200EF2FFFEE33FECD33CDCC94
:10062D0033CCC58233C5829BED9AEC99E582984017
:10063D000CF582EE9BFEED9AFDEC99FC0FD5F0D6F4
:10064D00E4CEFBE4CDFAE4CCF9A88222B800C1B91E
:10065D000059BA002DEC8BF084CFCECDFCE5F0CB5C
:10066D00F97818EF2FFFEE33FEED33FDEC33FCEB95
:10067D0033FB10D703994004EB99FB0FD8E5E4F950
:10068D00FA227818EF2FFFEE33FEED33FDEC33FC3D
:10069D00C933C910D7059BE99A4007EC9BFCE99A31
:1006AD00F90FD8E0E4C9FAE4CCFB2275F010EF2F76
:1006BD00FFEE33FEED33FDCC33CCC833C810D70776
:1006CD009BEC9AE899400AED9BFDEC9AFCE899F8B1
:0E06DD000FD5F0DAE4CDFBE4CCFAE4C8F92244
:0E06EB00C3E49FFFE49EFEE49DFDE49CFC2220
:1006F900EB9FF5F0EA9E42F0E99D42F0E89C45F057
:0107090022CD
:0C070A00ECF0A3EDF0A3EEF0A3EFF02262
:10097F008B568A578958E4F562F561F560F55FF596
:10098F005DF55EE55A455B45596012EBC0E0EAC084
:10099F00E0E9C0E0AB59AA5AA95B120765AB56054F
:1009AF0058E558AA577002055714F91205D7F56381
:1009BF00C394094007E563D3940D40E1E5636420D8
:1009CF0060DBE563B42D05435E038016E563B42B4E
:1009DF0005435E01800C74FF2558F55874FF355799
:1009EF00F557E55C60046410703FAB56AA57A958E1
:1009FF001205D764306009E55C702E755C0A80299A
:100A0F009000011205F0FF64786004EFB4581343AF
:100A1F005E01755C1074022558F558E43557F5578B
:100A2F008007E55C7003755C08AB560558E558AA5E
:100A3F00577002055714F91205D7F563C394614037
:100A4F000AE563D3947A50035363DF74D02563F5BB
:100A5F0063C3940A400CE5639411406D74F92563E8
:100A6F00F563E563D3955C5060435E0185626785EE
:100A7F006166856065855F64AF5C7E00E4FCFDABFD
:100A8F0062AA61A960A85F120716C8ECC8C9EDC9B0
:100A9F00CAEECACBEFCBE4FCFDFEEB2563F562EEAD
:100AAF003AF561ED39F560EC38F55FAF62AE61ADE7
:100ABF0060FCAB67AA66A965A864D31206F9500358
:100ACF00020A38435E04020A38E55E20E003E48040
:100ADF002DE55A455B4559601EAB56E55824FFF985
:100AEF00E55734FFFAEBC0E0EAC0E0E9C0E0AB59EC
:100AFF00AA5AA95B120765E55E30E20774FFFFFE95
:100B0F00FDFC22E55EAF62AE61AD60AC5F30E1032C
:040B1F000206EB22BD
:10157700020036E493A3F8E493A34003F68001F254
:1015870008DFF48029E493A3F85407240CC8C33375
:10159700C4540F4420C8834004F456800146F6DF44
:1015A700E4800B01020408102040809019DFE47EDC
:1015B700019360BCA3FF543F30E509541FFEE49339
:1015C700A360010ECF54C025E060A840B8E493A300
:1015D700FAE493A3F8E493A3C8C582C8CAC583CA2B
:1015E700F0A3C8C582C8CAC583CADFE9DEE780BEE3
:0119F70000EF
:10071600E88FF0A4CC8BF0A42CFCE98EF0A42CFC82
:100726008AF0EDA42CFCEA8EF0A4CDA8F08BF0A400
:100736002DCC3825F0FDE98FF0A42CCD35F0FCEB5F
:100746008EF0A4FEA9F0EB8FF0A4CFC5F02ECD3924
:0F075600FEE43CFCEAA42DCE35F0FDE43CFC2291
:10076500BB011A89828A83D0F0D0E0F8D0E0F9D0B5
:10077500E0FAD0E0FBE8C0E0C0F00207BD5016E9A2
:10078500F8D083D082D0E0F9D0E0FAD0E0FBC08287
:10079500C0830207B4BBFE16E9F8D083D082D0E04F
:0F07A500F9D0E0FAD0E0FBC082C0830207C62281
:0907B400EBF608EAF608E9F6226A
:0907BD00EBF0A3EAF0A3E9F0223D
:0907C600EBF208EAF208E9F22264
:00000001FF
